:103C96000FC30FBF0FBB0FB60FB20FAC0FA70FA10D
:103CA6000F9B0F950F8E0F870F800F780F700F6881
:103CB6000F5F0F550F4B0F410F360F2B0F1F0F12B4
:103CC6000F060EF80EEA0EDB0ECC0EBC0EAB0E9AED
:103CD6000E880E750E620E4E0E390E240E0E0DF760
:103CE6000DDF0DC70DAE0D940D790D5E0D410D2442
:103CF6000D070CE80CC90CA90C890C680C460C23A2
:103D06000C000BDC0BB80B930B6E0B480B210AFA5D
:103D16000AD30AAC0A840A5B0A330A0A09E109B71C
:103D2600098E0965093B091108E808BE0895086C63
:103D36000842081907F107C807A00778075007299E
:103D4600070206DB06B5068F066A0645062105FD4F
:103D560005DA05B70595057405530532051204F312
:103D660004D404B60498047B045F04430428040DB9
:103D760003F303DA03C103A90391037A0363034D33
:103D860003370322030E02F902E602D302C002AE93
:103D9600029C028B027A026A025A024B023C022DF4
:103DA600021F0211020301F601E901DD01D001C57E
:103DB60001B901AE01A30198018E0184017A017156
:103DC6000168015F0156014D0145013D0135012E96
:103DD6000126011F01180111010B010400FE00F864
:103DE60000F200EC00E600E100DC00D600D100CCD9
:103DF60000C800C300BE00BA00B600010C010104F1
:103E060002011E030A960401320502020600640737
:103E1600010108000009015A0E01010F00011200FC
:103E26006413010114013C1501FA1664FA17FFFF29
:103E36001D00072000072400022701012F013C3046
:103E4600FFFF32010335FFFF3603073CFFFF3DFF4F
:103E5600FF180002191E461A00021B00022D32C866
:103E66002E0001FAFAFA18000019FFFF1A00001BCB
:0B3E760000002D32C82E0001FAFAFAFD
:10004800900786E0FEA3E0FF7457BE0010D39F40E0
:100058000C903E0012001EE493F599802F90001436
:10006800E0D394044014900786E0FEA3E0FF903E9E
:100078000012001EE493F5998012900786E0FEA313
:10008800E0FF903E1512001EE493F5999007861242
:10009800000E900786E0FEA3E0FF746C6F4E7003BD
:1000A80075130022900072E0B40208740190007287
:1000B800F0D20C90013AE090002AF090013BE090D9
:1000C800002BF090013CE090002CF0A20AB34016FF
:1000D80090013AE0700C90013BE0700690013CE022
:1000E80060028002C20A90013AE0B4300F90013BEE
:1000F800E0B4470890013CE0643B60028004D20B06
:100108008002C20BE558B40102800302022E90005F
:1001180057E0F565900062E0F567900063E0F568E8
:10012800900074E0F56990007AE0900029F0900062
:100138007CE0F56490007DE0F566900080E0F56372
:10014800900081E0F562900090E0900041F090000E
:1001580091E0900042F0900092E0900043F090000F
:1001680093E0900044F0900094E0900045F09000F7
:1001780095E0900046F0900096E0900047F09000DF
:1001880097E0900048F0900099E0900033F09000DC
:100198009AE0900034F090009BE0900035F09000D9
:1001A8009CE0900036F0900079E0B4011790000AC6
:1001B800740FF0A374FFF090000CE4F0A3F0740245
:1001C800900079F0900079E0B4035990000CE0FEBB
:1001D800A3E0FF90000AE0FCA3E0FD120003741006
:1001E800123FE17408123FD3EF900026F0EF70063B
:1001F80074FF900026F07400900079F090000BE0F6
:10020800900027F090000AE0900028F0900026E087
:10021800900789F0900027E090078AF0900028E086
:1002280090078BF0803F900081E07006755801754B
:100238006200A20AB3402E90013AE090002AF090A2
:10024800013BE090002BF090013CE090002CF090F6
:10025800002AE0700C90002BE0700690002CE06003
:10026800028002C20AE5657003756502E5677003DE
:100278007567027E867F64E5658E048F05FF123FF1
:10028800C38C398D3AE56875F0FAA4FFAEF0E567DE
:100298008E048F05FF123FC38C3D8D3E90004FE0CA
:1002A800F55F90004DE0FE900069E0B506189000FB
:1002B8004CE0FE900068E0B5060C90004BE0FE9024
:1002C8000059E06E606F900069E07006900068E089
:1002D80060067400900059F0900069E0B40208903C
:1002E80000497401F08005900049E4F0900068E04E
:1002F800B4020890004A7401F0800590004AE4F0C6
:10030800900068E0600690004AE060028005755F32
:10031800038003755F04E559B55802D20C90006854
:10032800E090004CF0900069E090004DF09000598A
:10033800E090004BF0740090009EF0740190009FD4
:10034800F074009000A0F074009000A1F074009088
:1003580000A2F074009000A3F074009000A4F07460
:10036800009000A5F074009000A6F074009000A71B
:10037800F074009000A8F074009000A9F074009048
:1003880000AAF074009000ABF074009000ACF07418
:10039800019000ADF074009000AEF074009000AFD2
:1003A800F074009000B0F074009000B1F074009008
:1003B80000B2F07400900362F07401900363F0746B
:1003C80001900364F07400900365F0740090036674
:1003D800F07400900367F07400900368F074019063
:1003E80003A2F074009003A3F074019003A4F074C6
:1003F800009003A5F074009003A6F074009003A782
:10040800F074009003A8F074009003E2F074009078
:1004180003E3F074009003E4F074009003E5F074D3
:10042800009003E6F074009003E7F074009003E88E
:10043800F07400900422F07400900423F07400908B
:100448000424F07401900425F07400900426F074DC
:1004580000900427F07400900428F022E5B554F7C2
:10046800F5B5E5B554FDF5B5C2A2C2A1C292C20761
:10047800E5B554FBF5B5755104E55104F552900006
:100488004FE0F55F900025E4F0C209E5B554FEF5AC
:10049800B5C28E758D00758B00754C00752600757C
:1004A8002500D28E22750A00750900AE09AF0A74BC
:1004B80057BE00039F500302056A903E0012001EBB
:1004C800E49390004E123FF90FBF00010EE0FC903C
:1004D8003E0012001EECFEE493FFEEC39F5026AED2
:1004E80009AF0A0FBF00010E903E0012001EAE09B0
:1004F800AF0AE493FC903E0012001EE49390004E75
:10050800123FF9ECF0AE09AF0A903E0012001EE46B
:100518009390004E123FF9E0FC903E0212001EEC50
:10052800FCE493FDECD39D4019903E0212001EE4BA
:1005380093FC903E0012001EE49390004E123FF987
:10054800ECF0AE09AF0A74022FFF50010E8E098F2E
:100558000A780A740126F6500418E436F6400302B5
:1005680004B322750A00750900AE09AF0A7415BEF6
:1005780000039F5003020638903E5712001EE49372
:1005880090004E123FF90FBF00010EE0FC903E575D
:1005980012001EECFEE493FFEEC39F5026AE09AF97
:1005A8000A0FBF00010E903E5712001EAE09AF0A97
:1005B800E493FC903E5712001EE49390004E123FC5
:1005C800F9ECF0AE09AF0A903E5712001EE4939082
:1005D800004E123FF9E0FC903E5912001EECFCE47C
:1005E80093FDECD39D4019903E5912001EE493FCF4
:1005F800903E5712001EE49390004E123FF9ECF023
:10060800AE09AF0A740F6F4E7006750A15750900AA
:10061800AE09AF0A74022FFF50010E8E098F0A78B7
:100628000A740126F6500418E436F64003020571F0
:1006380022750A00750900AE09AF0A7415BE0003D9
:100648009F5003020706903E6C12001EE493900030
:100658004E123FF90FBF00010EE0FC903E6C1200F5
:100668001EECFEE493FFEEC39F5026AE09AF0A0FBF
:10067800BF00010E903E6C12001EAE09AF0AE49353
:10068800FC903E6C12001EE49390004E123FF9EC71
:10069800F0AE09AF0A903E6C12001EE49390004E33
:1006A800123FF9E0FC903E6E12001EECFCE493FD54
:1006B800ECD39D4019903E6E12001EE493FC903ED0
:1006C8006C12001EE49390004E123FF9ECF0AE0954
:1006D800AF0A740F6F4E7006750A15750900AE09DA
:1006E800AF0A74022FFF50010E8E098F0A780A7420
:1006F8000126F6500418E436F6400302063F2205A8
:100708004D22054C22054EC2CF2290F800E4936496
:1007180006600280FE75840175A70075FF8090074A
:1007280088E4F075C91075A70F75A1C775A700757E
:10073800D90075CEFF75A70F75F1FE75F2FF75F339
:100748003775F47875A4BA75A5FF75A60775AE0058
:1007580075AFFF75D48175D5FF75D6FF75D7FFC204
:1007680096C295C2A0C297E5B554BFF5B5E5B55494
:10077800DFF5B5E5B554EFF5B5E5B5547FF5B5E565
:10078800B554F7F5B5E5B554FDF5B575A70075A2EF
:100798000175A14775F80975BC0175BE0475BD6C76
:1007A80075BE0775BDA075BE0875BD0175BC007521
:1007B800BB1875BC2075BA0875E88075D11375A784
:1007C8000F75E10575E20075C7407597007597804C
:1007D800740A123FB37597C0E5975420700280F8E9
:1007E800758F0275A700D2AF75980075A90C75A70B
:1007F8000F75AB4375ADFB75AC1E75A700758911F8
:10080800758E00758C00758A00D2A9D28C758D0002
:10081800758B00D2ABD28E75CD0075CC0075CA0031
:1008280075CB00D2ADC2CFD2CA759104759200754E
:1008380093CD75EF0675D94075CF01900786E4F022
:10084800A3F0751300751400C299D20AC20D1204E0
:100858006474C8F5187517001225C575A70FE5FB50
:1008680090001AF0E5FA90001BF0E5F990001CF0F2
:1008780075A70090F800E493F5081226FC122C36B0
:10088800900789E0900026F090078AE0900027F012
:1008980090078BE0900028F090078CE0900029F0FA
:1008A80090078DE0F56590078EE0F56790078FE07B
:1008B800F568900790E0F569900791E0F564900776
:1008C80092E0F566900793E0F563900794E0F5628F
:1008D800900795E090002AF0900796E090002BF0A2
:1008E800900797E090002CF0900798E0900041F076
:1008F800900799E0900042F090079AE0900043F04A
:1009080090079BE0900044F090079CE0900045F031
:1009180090079DE0900046F090079EE0900047F019
:1009280090079FE0900048F09007A0E0900033F017
:100938009007A1E0900034F09007A2E0900035F015
:100948009007A3E0900036F07400900082F09001C8
:100958003AE0700C90013BE0700690013CE06002C8
:100968008004C20A8002D20A90F807E4939000211A
:10097800F0900021E0440A900021F0900021E0541A
:10098800FE900021F07406900012F074029000139B
:10099800F090F802E493900014F07403900015F0BE
:1009A8007403900016F0742A900017F074059000F4
:1009B80018F0900014E0B404067404900018F07461
:1009C80005900019F090F804E49390001DF074006D
:1009D80090001EF090F805E49390001FF090F80640
:1009E800E493900020F074FF900022F0745390017B
:1009F80025F07475900126F0747A900127F07475CB
:100A0800900128F0746B900129F0746990012AF024
:100A1800742090012BF0744790012CF074319001F0
:100A28002DF0743390012EF0742090012FF074345F
:100A3800900130F07453900131F07470900132F0ED
:100A48007464900133F090007AE0D3940140067406
:100A58000090007AF0755801755901740390004CA4
:100A6800F01200AC1204AD900014E0B404051206B4
:100A780039800312056B1225F1E5B554FEF5B590E2
:100A88000025E4F0900786E4F0A3F07524007523B0
:100A980000754800752A00752900754900753200EF
:100AA800753100754A00755400755500755A007502
:100AB800510475520175343C753300756F00756EBD
:100AC800007570CD75560075570075430075440064
:100AD800754500754600755B0075470075420075E1
:100AE8004100900006E4F0A3F0900008E4F0A3F0C1
:100AF800755D00755E0090000E74FDF0A374E8F05B
:100B0800900023E4F07464900024F0C200D201C283
:100B180002D203754D00756C00C294C293C287C29D
:100B280090C291C20C7E017F00900028E0123FE144
:100B3800900027E02FFF50010E90000AEEF0A3EF7F
:100B4800F0900026E0700674FF900026F090000AEE
:100B5800E0FEA3E0FFEFD394FFEE940F4007900070
:100B68000AE4F0A3F07400900071F074009000792A
:100B7800F07400900082F0740090008DF074009082
:100B880000B4F0E5667003756604743A90074EF099
:100B980074FD90074FF09003D4E0900414F0D2B0A5
:100BA800D2B7D2A7D2A6D2B1D2A3C207A2B6B39265
:100BB80004A2B3B39205D29CD2EC75CF01A298B32C
:100BC8004005C298122F9AE5136006A299B3B34064
:100BD800028005C29912350AE51464016005E5141E
:100BE800B4040280D5E54DD39405400CE55AC3946E
:100BF800C85002055A754D00E570C394F0501A7834
:100C08006E12003FAE6EAF6FEFD394E8EE940340E0
:100C1800080570756F00756E00C28E7E047F00E552
:100C28004C123FE1E58D75F004A4FDACF0EF2DFD0D
:100C3800EE3CFCE58B75F04084FF7E00ED2FFFEC69
:100C48003EFE8E258F26D28EA2B6300401B3500305
:100C5800020D95A2B6300401B35003020D95A2B659
:100C680040670554A20D400575FFA0D20DE5B544B7
:100C780001F5B5900024E4F0E554D3956540487C2F
:100C8800867D64AE25AF26123E818E238F24E548EB
:100C98002FFF50010E7401123FD38E238F24852419
:100CA80048755401C28E758D00758B00754C00D245
:100CB8008E7403BE00039F50069000257401F0E572
:100CC80043B40603754300D204A2B6B35003020D21
:100CD80095C20490006BE0601812364BA200B34036
:100CE80008E5B54408F5B58006E5B554F7F5B580CF
:100CF80002C20090006EE060181237A0A202B34052
:100D080008E5B54402F5B58006E5B554FDF5B580AE
:100D180006E5B554FDF5B5A207B34004D2878002B5
:100D2800C287900059E06004D2908002C29090007F
:100D38004AE0B40104D2948002C294900049E0B41D
:100D48000104D2938002C293A209B34004D29180D5
:100D580002C291900018E0FE900014E0C39E400982
:100D6800900014E0D39408400974FB900023F0121B
:100D7800046490001DE0601590001DE0FE900017CF
:100D8800E06E600974FE900023F0120464C2CA7E0B
:100D9800017F00E54E123FE1E5CD2FFF50010E8E99
:100DA800278F28D2CAE564B4014890000EE0FCA35E
:100DB800E0FDEFC39DEE9C4039B208E52A45296065
:100DC80013A208B34008E5B54404F5B58006E5B5B7
:100DD80054FBF5B590000EE0FEA3E0FF900010E094
:100DE800FCA3E0FDEF2DFDEE3CFC90000EECF0A323
:100DF800EDF0A2B3300501B35003020EE3A2B33005
:100E08000501B35003020EE3A2B35003020EDC0542
:100E180055A20D400575FFA0D20DE5B54401F5B505
:100E2800900024E4F0E555D395675003020EDA7C70
:100E3800EA7D60AE27AF28123E818E298F2AE568A9
:100E4800123FE174FF8E048F05FF123FC38C298D7A
:100E58002AE5492DFD50010C74018C068D07123FBF
:100E6800D38E298F2A852A49A209B34015746412A2
:100E78003FE1900067E08E048F05FF123FC38C2985
:100E88008D2A75550190000EE0FEA3E0FFAC27AD5A
:100E98002812000390000EEEF0A3EFF0E566FF12B3
:100EA8003FC3740AFF123FC390007BE08C068D0796
:100EB800123FE174148E048F05FF123FC390001097
:100EC800ECF0A3EDF0C2CA75CD0075CC00754E00EC
:100ED800D2CAD205A2B3B34002C205900025E0B43D
:100EE8000107E556C3940640030214F4E56C902507
:100EF800A4F8282873900059E0C394024003021014
:100F080051E551D394015003021051E55175F04059
:100F1800A4FFAEF090031212001EE0C395455018CE
:100F2800E55175F040A4FFAEF090031112001EE0E9
:100F3800F52E752D00021051E55175F040A4FFAE55
:100F4800F090031012001EE0C395454003020FED18
:100F5800E55175F040A4FFAEF090031112001EE5B4
:100F68005175F040A4FFAEF0E0FC90030F12001E94
:100F7800ECFEE0FFEEC39FFEE5518E0475F040A441
:100F8800FFAEF090031012001EE0F40425458C001B
:100F980088F0A4FFAEF0E5518F048E0575F040A4EB
:100FA800FFAEF090031212001EE55175F040A4FF49
:100FB800AEF0E0FA90031012001EEAFEE0FFEEC366
:100FC8009FFECDCCCD8E07123FC3E55175F040A4EE
:100FD800FFAEF090030F12001EE02DFD50010C8CA7
:100FE8002D8D2E8064E55175F040A4FFAEF090037E
:100FF8000F12001EE55175F040A4FFAEF0E0FC9022
:10100800030E12001EECFEE0FFEEC39F8545F0A420
:10101800FFAEF0E5518F048E0575F040A4FFAEF0E9
:1010280090031012001EE0FECDCCCD8E07123FC3F8
:10103800E55175F040A4FFAEF090030E12001EE0DB
:101048002DFD50010C8C2D8D2E756C010214F49021
:101058000059E0C39402400302120490004FE0D309
:10106800955150030211ADE55175F040A4FFAEF063
:1010780090031812001EE0C395455018E55175F00D
:1010880040A4FFAEF090031712001EE0F52C752B5C
:10109800000211ADE55175F040A4FFAEF0900316C3
:1010A80012001EE0C395454003021149E55175F051
:1010B80040A4FFAEF090031712001EE55175F040F2
:1010C800A4FFAEF0E0FC90031512001EECFEE0FF5A
:1010D800EEC39FFEE5518E0475F040A4FFAEF0907C
:1010E800031612001EE0F40425458C0088F0A4FFC6
:1010F800AEF0E5518F048E0575F040A4FFAEF09078
:10110800031812001EE55175F040A4FFAEF0E0FA96
:1011180090031612001EEAFEE0FFEEC39FFECDCC40
:10112800CD8E07123FC3E55175F040A4FFAEF09095
:10113800031512001EE02DFD50010C8C2B8D2C8008
:1011480064E55175F040A4FFAEF090031512001E3F
:10115800E55175F040A4FFAEF0E0FC9003141200D6
:101168001EECFEE0FFEEC39F8545F0A4FFAEF0E560
:10117800518F048E0575F040A4FFAEF0900316124F
:10118800001EE0FECDCCCD8E07123FC3E55175F0B1
:1011980040A4FFAEF090031412001EE02DFD500194
:1011A8000C8C2B8D2CE551B40122E55FD3940140C2
:1011B8001BE551C395565014E545C39405500D9051
:1011C800035FE0A829B80006952A400280037551FC
:1011D80002E551B55F2290004FE0D395514019E5E3
:1011E8005175F040A4FFAEF090031712001EE0A85E
:1011F80023B80006952440028002055F756C020240
:1012080014F4900059E0B4022AE55175F040A4FFA7
:10121800AEF090031712001EE0F52C752B00E55177
:1012280075F040A4FFAEF090030E12001EE0F52EFC
:10123800752D00900059E0B4030F900051E0F52C93
:10124800752B00752E00752D00756C030214F4E5DE
:101258005175F040A4FFAEF090032012001EE0C3C9
:10126800955A400302132B900049E07036E551D39C
:1012780094014029AE23AF24AC2DAD2EEDD39FECC5
:101288009E401AE55175F040A4FFAEF090031E127F
:10129800001EE0A829B80005D3952A50028002153F
:1012A800518034E551D394024029AE23AF24AC2DAC
:1012B800AD2EEDD39FEC9E401AE55175F040A4FF8A
:1012C800AEF090031E12001EE0A829B80005D395C1
:1012D8002A500280021551E551B55236E551C395A1
:1012E8005F502FE551C395565028AE23AF24AC2B41
:1012F800AD2CEFD39DEE9C4019E55175F040A4FF4D
:10130800AEF090031F12001EE0A829B80006952A27
:10131800400280020551C292E55165526005C2073C
:10132800755A00756C040214F4E55175F040A4FF79
:10133800AEF090031A12001EE0B40117E55175F0E3
:1013480040A4FFAEF090032012001EE0240AC395CB
:101358005A4003021401753064752F00A207B35078
:101368000B900060E02405C395454003021401E595
:101378005175F040A4FFAEF090031D12001EE0C3AB
:1013880095454064E55175F040A4FFAEF090031C0C
:1013980012001EE55175F040A4FFAEF0E0FC90038A
:1013A8001B12001EECFEE0FFEEC39F8545F0A4FF74
:1013B800AEF0E5518F048E0575F040A4FFAEF090B5
:1013C800031D12001EE0FECDCCCD8E07123FC3E5F3
:1013D8005175F040A4FFAEF090031B12001EE02DE3
:1013E800FD50010C8C2F8D30AE23AF24AC2FAD30C7
:1013F800EFD39DEE9C4002D207756C050214F4E50C
:1014080051B40109900059E0C3940240030214D476
:10141800900358E0D3954550030214D4900356E046
:10142800C395455040900357E0FE900355E0F404FF
:101438002EFE900356E0F40425458E0088F0A4FFA4
:10144800AEF0900358E0FC900356E0F4042C8E04B0
:101458008F05FF123FC3900355E02DFD50010C8C02
:101468002B8D2C802C900355E0FE900354E0F4045F
:101478002E8545F0A4FFAEF0900356E08E048F054C
:10148800FF123FC3900354E02DFD50010C8C2B8DAF
:101498002CE551C3955F502FE551C395565028AEA2
:1014A80023AF24AC2BAD2CEFD39DEE9C4019E55116
:1014B80075F040A4FFAEF090031F12001EE0A829AB
:1014C800B80006952A40028003755102900049E051
:1014D800B40106E551640160028003755102E551CB
:0C14E80065526005C207755A00756C0063
:1025A400020EFD02105702120A02125702133102E0
:0225B40014070A
:1014F400900050E02402A823B80007D395244002AA
:10150400C207900025E0B40109900059E0C3940398
:10151400400302167A900049E060030215CAE551BF
:10152400D394014034E55175F040A4FFAEF090032C
:101534001412001EE0A823B8001FD39524401AE516
:101544005175F040A4FFAEF090031F12001EE0A8F6
:1015540029B80005D3952A500280021551E551D3CC
:101564009401402FE55175F040A4FFAEF0900312B2
:1015740012001EE0C39545501AE55175F040A4FFD2
:10158400AEF090031E12001EE0A829B80005D39502
:101594002A500280021551E551D394014021E551AE
:1015A400D39556401AE55175F040A4FFAEF0900370
:1015B4001E12001EE0A829B80005D3952A50028007
:1015C40002155102166FE551D394024034E551756A
:1015D400F040A4FFAEF090031412001EE0A823B85C
:1015E400001FD39524401AE55175F040A4FFAEF0D6
:1015F40090031F12001EE0A829B80005D3952A50B5
:101604000280021551E551D39402402FE55175F043
:1016140040A4FFAEF090031212001EE0C3954550A3
:101624001AE55175F040A4FFAEF090031E12001E9F
:10163400E0A829B80005D3952A500280021551E587
:1016440051D394024021E551D39556401AE5517582
:10165400F040A4FFAEF090031E12001EE0A829B8CB
:101664000005D3952A500280021551E55165526058
:1016740005C207755A00900060E0D3954550099063
:101684000054E0C395455002C207900059E070032E
:101694000218DDA2A5B34008A2A4B340030218C6F1
:1016A400AE35AF367441D39F749C9E400578351295
:1016B400003FAE35AF36EFB48806EEB413028003B4
:1016C4000218A3A2A55003021766900059E0B401C2
:1016D4000B90004FE0D3955F4002055F900059E006
:1016E400B40253E55175F040A4FFAEF0900320120C
:1016F400001EE0C3955A503E90004FE0D3955140F0
:1017040020E551C395565019E55175F040A4FFAE3C
:10171400F090031412001EE0A823B800069524409C
:10172400028002055190004FE0F55FE5516552607B
:1017340005C207755A00900059E0B4032590004F84
:10174400E0D395514007E551C39556400280020508
:101754005190004FE0F55FE55165526005C2077591
:101764005A00A2A450030218A3900059E0B4016ED9
:10177400900049E07035E551D394014029E5517555
:10178400F040A4FFAEF090031E12001EE0A829B89A
:10179400000FD3952A400A1551755A0085515F8070
:1017A4000385515F8003755F018033E551D3940253
:1017B4004029E55175F040A4FFAEF090031E1200DD
:1017C4001EE0A829B8000FD3952A400A1551755A6E
:1017D4000085515F800385515F8003755F0290002F
:1017E40059E0D394015003021897E55175F040A4D1
:1017F400FFAEF090032012001EE0C3955A4003028E
:101804001897900049E07041E551D394014034E5C4
:101814005175F040A4FFAEF090031112001EE0A831
:1018240023B8001FD39524401AE55175F040A4FF56
:10183400AEF090031E12001EE0A829B80005D3954F
:101844002A500280021551803FE551D3940240345E
:10185400E55175F040A4FFAEF090031112001EE0B4
:10186400A823B8001FD39524401AE55175F040A46D
:10187400FFAEF090031E12001EE0A829B80005D3A5
:10188400952A500280021551E55165526005C20740
:10189400755A00E556B40704055D8003755D00E5DF
:1018A40062B4010EAE35AF36EF64407005EE649C51
:1018B4006002800EA2A54003755801A2A4400375DE
:1018C4005802A2A5B3B35006A2A4B3B34002800643
:1018D4007536007535000219CBA2A5B34008A2A441
:1018E400B340030219B7AE35AF367441D39F749C2D
:1018F4009E4005783512003FAE35AF36EFB488060A
:10190400EEB4130280030219B7A2A5406F900068D9
:10191400E0605A90004AE0B4010790004AE4F08085
:101924000690004A7401F090004AE07005755F0368
:101934008003755F0490004AE0B40104D2948002ED
:10194400C294E551B4041AE55175F040A4FFAEF019
:1019540090031E12001EE0A829B80005D3952A5052
:10196400028008755103C207755A008003755F042D
:10197400E556B40704055D8003755D00A2A44033F9
:10198400900069E06021900049E0B40107900049AB
:10199400E4F080069000497401F0900049E0B4013D
:1019A40004D2938002C293E556B40704055D800314
:1019B400755D00A2A5B3B35006A2A4B3B3400280E0
:1019C40006753600753500E5586559600690008245
:1019D400E06003021B53C29C751400751300C2CA55
:1019E400E5589025B6F82828738012122C36800DFD
:0D19F400122D0F8008122DE88003122EC165
:0F25B6000219ED0219EF0219F40219F90219FEC8
:101A0100900029E090007AF0E565900057F0E567D5
:101A1100900062F0E568900063F0E569900074F071
:101A2100E56490007CF0E56690007DF0E563900050
:101A310080F0E562900081F090002AE090013AF098
:101A410090002BE090013BF090002CE090013CF0E5
:101A5100900041E0900090F0900042E0900091F001
:101A6100900043E0900092F0900044E0900093F0E9
:101A7100900045E0900094F0900046E0900095F0D1
:101A8100900047E0900096F0900048E0900097F0B9
:101A9100900033E0900099F0900034E090009AF0CB
:101AA100900035E090009BF0900036E090009CF0B3
:101AB1007400900082F07453900125F074759001C8
:101AC10026F0747A900127F07475900128F0746BF8
:101AD100900129F0746990012AF0742090012BF093
:101AE100744790012CF0743190012DF07433900102
:101AF1002EF0742090012FF07434900130F0745363
:101B0100900131F07470900132F07464900133F0FF
:101B11009003D4E0900414F0743A90074EF074FDF1
:101B210090074FF01200AC900004E4F0A3F0900095
:101B3100067475F0A37430F09000087475F0A37406
:101B410030F0855859D2CA754C00D29C741B900054
:101B510023F0E556C394065005E551B55203021B27
:101B6100E2C207E55175F040A4FFAEF090032212E6
:101B7100001EE030E003D38001C39296E55175F079
:101B810040A4FFAEF090032312001EE030E003D327
:101B91008001C39295E55175F040A4FFAEF090032A
:101BA1002412001EE030E003D38001C392A0E5516E
:101BB10075F040A4FFAEF090032512001EE030E066
:101BC10003D38001C39297855152AE29AF2A740580
:101BD100BE00039F5007E545D3940550028002D211
:101BE10092E556D394055003021D2FC207E551D348
:101BF10094015003021C84E55175F040A4FFAEF03E
:101C010090031E12001EE0A829B80007D3952A40B0
:101C1100021551E55165526067E55175F040A4FF29
:101C2100AEF090032212001EE030E003D38001C326
:101C31009296E55175F040A4FFAEF0900323120097
:101C41001EE030E003D38001C39295E55175F04069
:101C5100A4FFAEF090032412001EE030E003D38015
:101C610001C392A0E55175F040A4FFAEF0900325A9
:101C710012001EE030E003D38001C39297855152D8
:101C8100021D2FE556B406349000ACE030E003D3DA
:101C91008001C392969000ADE030E003D38001C390
:101CA10092959000AEE030E003D38001C392A09002
:101CB10000AFE030E003D38001C39297E556B4074B
:101CC100349000A5E030E003D38001C392969000E8
:101CD100A6E030E003D38001C392959000A7E030E5
:101CE100E003D38001C392A09000A8E030E003D3C9
:101CF1008001C39297E556B4083490009EE030E02D
:101D010003D38001C3929690009FE030E003D3801B
:101D110001C392959000A0E030E003D38001C3920B
:101D2100A09000A1E030E003D38001C39297A20705
:101D3100B34005E556B407037570CDE595C39570BD
:101D41004004C2A18002D2A1E543C394064003022C
:101D5100234CA2EDB3500302234CC2EDE5436003D3
:101D6100021EAE7E017F00E5BE123FE1E5BD2FFF01
:101D710050010E900000EEF0A3EFF0900029E0B4C6
:101D810001177E0F7FFF900000E0FCA3E0FD120031
:101D910003900000EEF0A3EFF0900079E0B4025B55
:101DA100900000E0FEA3E0FF90000AE0FCA3E0FD4C
:101DB100EDD39FEC9E400F900000E0F8A3E090006F
:101DC1000AC8F0A3C8F0900000E0FEA3E0FF900075
:101DD1000CE0FCA3E0FDEFD39DEE9C400F900000D2
:101DE100E0F8A3E090000CC8F0A3C8F0900000E078
:101DF100FEA3E0FF7404123FD38F44900079E0709A
:101E010060900000E0FEA3E0FF90000AE0FCA3E088
:101E1100FDEFD39DEE9C400D120003900000EEF00B
:101E2100A3EFF08007900000E4F0A3F0900000E041
:101E3100FEA3E0FF7410123FE1900026E08E048FB4
:101E410005FF123FC3900000ECF0A3EDF07400D346
:101E51009D74019C4008900001E0F54480037544A5
:101E6100FFE54475F00AA4FFAEF074198E048F05E6
:101E7100FF123FC38D45ED2532FFAE3150010E7487
:101E810001123FD38F45854532753100EFD39462FE
:101E91004003754562900072E0640160069000663F
:101EA100E060028005754301800375BB17E543B40B
:101EB10001028003021F9E7E017F00E5BE123FE109
:101EC100E5BD2FFF50010E900000EEF0A3EFF09062
:101ED1000072E0B4017EE53445336025AC33AD34A6
:101EE1001DBDFF011C8F028E038C068D07903C9651
:101EF10012002EE493FE740193FFEFC39AEE9B4010
:101F0100028005783312400BAE33AF3474B3BE0098
:101F110025D39F4021900000E0FCA3E0FD0FBF000E
:101F2100010E903C9612002EE493FE740193FFED96
:101F3100C39FEC9E40028005783312003FAE33AF61
:101F410034E569123FE174648E048F05FF123FC3CB
:101F51008D478033900066E0602D900000E0FEA385
:101F6100E0FFEFD39400EE9408400F900066E0B4D8
:101F71000104C2098002D209800D900066E0B4011B
:101F810004D2098002C209900072E06402600690E6
:101F91000066E0600575BB168003754302E543B436
:101FA1000202800302208C7E017F00E5BE123FE128
:101FB100E5BD2FFF50010E900000EEF0A3EFF09071
:101FC1000072E0B4027EE53445336025AC33AD34B4
:101FD1001DBDFF011C8F028E038C068D07903B2CCB
:101FE10012002EE493FE740193FFEFC39AEE9B401F
:101FF100028005783312400BAE33AF3474B3BE00A8
:1020010025D39F4021900000E0FCA3E0FD0FBF001D
:10201100010E903B2C12002EE493FE740193FFED10
:10202100C39FEC9E40028005783312003FAE33AF70
:1020310034E569123FE174648E048F05FF123FC3DA
:102041008D478033900066E0602D900000E0FEA394
:10205100E0FFEFD39400EE9408400F900066E0B4E7
:102061000104C2098002D209800D900066E0B4012A
:1020710004D2098002C209900072E0700375470022
:10208100900066E07002C20975BB1FE543B40345C9
:102091007E017F00E5BE123FE1E5BD2FFF50010E3D
:1020A100900000EEF0A3EFF07409123FE174E68EA8
:1020B100048F05FF123FC38C418D42E54A2DFD502F
:1020C100010C74018C068D07123FD38E418F42851E
:1020D100424A75BB19E543B4040280030222347EEF
:1020E100017F00E5BE123FE1E5BD2FFF50010E90DB
:1020F1000000EEF0A3EFF07404123FD38F4BE563C1
:10210100B4010280030221C1756A00756A00E56AA3
:10211100D3940740030221AEE56A900041123FF9D2
:10212100E0D3954B501AE56A900041123FF9E0F473
:1021310004254BFEE56A900037123FF9EEF0801757
:10214100E56A900041123FF9E0C3954BFEE56A90C4
:102151000037123FF9EEF0E56AC39404400990009C
:1021610084E0C3956A503BE56A6029E56A900037CF
:10217100123FF9FEE0FFEE90003FE0D39F4013E5F0
:102181006A900037123FF9E090003FF0E56A900055
:1021910040F0800E900037E090003FF07400900016
:1021A10040F0786A740126F6400302210F90004046
:1021B100E0F4042408F556E556D394054002C29292
:1021C100E563D39401402FE54BD3946E4004D20EC6
:1021D1008002C20E755605E563B40205A20EB34036
:1021E100028003755607E563B40306A20EB3B3403C
:1021F100028003755607E55765566008E55104F5F9
:1022010052855657E556B40708E5B54480F5B580C3
:1022110006E5B5547FF5B5E55664066005E556B4A7
:102221000808E5B54410F5B58006E5B554EFF5B5F8
:1022310075BB13E543B4050280030223487E017F89
:1022410000E5BE123FE1E5BD2FFF50010E900000F9
:10225100EEF0A3EFF07404123FD38F46E562B402AF
:10226100028003022345756A00756A00E56AD3940A
:102271000340030222FCE56A900033123FF9E0D3E8
:102281009546501AE56A900033123FF9E0F40425AF
:1022910046FEE56A90002D123FF9EEF08017E56ADF
:1022A100900033123FF9E0C39546FEE56A90002D98
:1022B100123FF9EEF0E56A6029E56A90002D123FC0
:1022C100F9FEE0FFEE900031E0D39F4013E56A9004
:1022D100002D123FF9E0900031F0E56A900032F0F4
:1022E100800E90002DE0900031F07400900032F0EB
:1022F100786A740126F6400302226D900082E07034
:1023010043E52A45296036E558C39403500A9000F5
:1023110032E004C3940340028007900032E004F5E8
:1023210058E558D39402400A900032E004D3940255
:1023310050028007900032E004F558800790003287
:10234100E004F55875BB180543D2ECE55DD3940460
:10235100500302246475CF01AE35AF367488D39F24
:1023610074139E4005A2A5B34014AE35AF367488F0
:10237100D39F74139E4005A2A4B3400280487835D0
:1023810012003FAE35AF36EFB4883BEEB41337A23F
:10239100A5B3500990004FE0D39551500280040538
:1023A100518011A2A5B3500890004FE06551600221
:1023B1008002D207A2A4B35007E551D39401500281
:1023C10080041551C207A2A5B3B35006A2A4B3B3AA
:1023D10040028006753600753500E551655260672B
:1023E100E55175F040A4FFAEF090032212001EE00B
:1023F10030E003D38001C39296E55175F040A4FF0C
:10240100AEF090032312001EE030E003D38001C33D
:102411009295E55175F040A4FFAEF09003241200AF
:102421001EE030E003D38001C392A0E55175F04076
:10243100A4FFAEF090032512001EE030E003D3802C
:1024410001C39297855152A20740057570CD800353
:102451007570FFE595C395704004C2A18002D2A1B9
:10246100022356A20DB3500DAE25AF2674E8C39FCB
:1024710074039E4002800575FFA0D20DAE25AF26E4
:10248100EFD39420EE944E5003022578120464C2D7
:102491008E758D00758B00754C00D28EC207756FDD
:1024A10000756E007570CD7551047524007523009B
:1024B100755400755A00C287900059E06004D290AB
:1024C1008002C29090004AE0B40104D2948002C21A
:1024D10094900049E0B40104D2938002C293A2090E
:1024E100B34004D2918002C29190006BE060181257
:1024F100364BA200B34008E5B54408F5B58006E5C2
:10250100B554F7F5B58002C20090006EE060181274
:1025110037A0A202B34008E5B54402F5B58006E54F
:10252100B554FDF5B58006E5B554FDF5B590000E41
:1025310074FDF0A374E8F0E543B40603754300901D
:102541000025E4F0752600752500758D00758B005A
:10255100754C00900024E0C394035008900024E0DF
:1025610004F080067403900024F0900024E0B4038A
:1025710006E5B554FEF5B5AE27AF28EFD39410EEBE
:102581009427401CC2CA75CD0075CC007528007512
:102591002700D2CA754E00752A00752900755500AD
:0325A100020BC268
:103952000000010001320164019601960200021288
:1039620002240200020003000340038003C004009B
:103972000440048004C0050006000600060006009C
:10398200060006000600060000FF013101630195F2
:1039920001FF01FF0211022302FF02FF02FF033FA8
:1039A200037F03BF03FF043F047F04BF04FF05FF3F
:1039B20006FF06FF06FF06FF06FF06FF06FF06FFDD
:1039C2000FAA0FA50F9F0F9A0F940F8D0F870F80CD
:1039D2000F780F710F680F600F570F4E0F450F3B97
:1039E2000F300F250F1A0F0E0F020EF50EE80EDB29
:1039F2000ECC0EBE0EAE0E9F0E8E0E7D0E6C0E5AAD
:103A02000E470E340E200E0C0DF70DE20DCB0DB548
:103A12000D9D0D850D6D0D540D3A0D200D050CE912
:103A22000CCE0CB10C940C760C580C3A0C1B0BFB04
:103A32000BDB0BBB0B9A0B790B570B350B130AF1F4
:103A42000ACE0AAB0A870A640A400A1C09F809D49A
:103A520009B0098C09670943091F08FB08D608B297
:103A6200088E086A0846082307FF07DC07B907968D
:103A720007730751072F070D06EC06CA06AA068927
:103A820006690649062A060A05EC05CD05B0059227
:103A920005750558053C0520050504EA04CF04B563
:103AA200049C04820469045104390422040B03F4C3
:103AB20003DE03C803B2039D038903750361034D4B
:103AC200033B03280316030402F202E102D102C0FF
:103AD20002B002A0029102820273026502570249F9
:103AE200023C022F02220216020901FD01F201E646
:103AF20001DB01D001C601BB01B101A7019D019407
:103B0200018B018201790170016801600158015045
:103B12000148014101390132012B0125011E011821
:103B22000111010B010500FF00FA0FA60FA00F996A
:103B32000F920F8B0F840F7C0F740F6B0F620F5855
:103B42000F4E0F430F380F2C0F1F0F120F050EF7DA
:103B52000EE80ED80EC80EB70EA50E930E800E6C90
:103B62000E580E420E2C0E150DFD0DE40DCB0DB1AF
:103B72000D950D790D5D0D3F0D200D010CE10CC071
:103B82000C9E0C7C0C590C350C100BEA0BC40B9ED2
:103B92000B760B4F0B260AFD0AD40AAA0A800A5595
:103BA2000A2A09FF09D409A8097C0950092508F93C
:103BB20008CD08A10875084A081E07F307C8079D23
:103BC20007730749072006F706CE06A6067E0657A4
:103BD2000630060A05E405BF059B05770554053244
:103BE200051004EF04CE04AE048F047104530435AF
:103BF200041903FD03E203C703AD0394037B0363CC
:103C0200034B0334031E030802F302DE02CA02B6A8
:103C120002A30291027F026D025C024C023C022C62
:103C2200021D020E020001F201E401D701CA01BE27
:103C320001B101A6019A018F0185017A0170016625
:103C4200015D0153014A014101390131012901217B
:103C520001190112010B010400FD00F700F000EA56
:103C620000E400DE00D900D300CE00C900C400BFCA
:103C720000BA00B500B100AD00A800A400A0009CED
:103C8200009900950091008E008A008700840081CF
:043C9200007E007B35
:1025C500751A00751900AE19AF1AAC17AD18EDC321
:1025D5009FEC9E401674FF123FB375CF01781A74B5
:1025E5000126F6500418E436F650DB22900786E4FF
:1025F500F0A3F0751000750F00751300751400C277
:102605000FD21022C2AF75D900758F0375B7A575A6
:10261500B7F190F800E4F0758F0175B7A575B7F1BE
:10262500E50890F800F075B7A575B7F190F801E4E5
:10263500F075B7A575B7F190079DE090F802F075B4
:10264500B7A575B7F19007A1E090F803F075B7A5A8
:1026550075B7F190079EE090F804F075B7A575B7CA
:10266500F190079FE090F805F075B7A575B7F19063
:1026750007A0E090F806F075B7A575B7F19007A229
:10268500E090F807F0758F0075D940D2AF2290071A
:1026950088E0B4AB61C2AF75D90075B62275F52275
:1026A500758F0375B7A575B7F1740090F600F075D1
:1026B5008F01750A00750900AE09AF0A7413BE00D3
:1026C500279F402475B7A575B7F190078912001E9D
:1026D500E0FC90F60012001EECF0780A740126F674
:1026E500500418E436F650D0758F0075F51175B69F
:1026F5002075D940D2AF22C2AF75D90075F52275C4
:102705000A00750900AE09AF0A7413BE00229F4086
:102715001F90F60012001EE493FC90078912001E1C
:10272500ECF0780A740126F6500418E436F650D514
:1027350075F51175D940D2AF22900788E0B4AA0289
:10274500800302287BC2AF75D90075B62275F522C4
:10275500758F0375B7A575B7F1740090EE00F07528
:10276500B7A575B7F1740090F000F075B7A575B70A
:10277500F1740090F200F075B7A575B7F17400908B
:10278500F400F0758F01750A00750900AE09AF0AEE
:1027950074FFC39F74019E402475B7A575B7F1906A
:1027A500004E12001EE0FC90EE0012001EECF078C8
:1027B5000A740126F6500418E436F650CF750A005F
:1027C500750900AE09AF0A74FFC39F74019E4024CA
:1027D50075B7A575B7F190024E12001EE0FC90F09A
:1027E5000012001EECF0780A740126F6500418E475
:1027F50036F650CF750A00750900AE09AF0A74FFA9
:10280500C39F74019E402475B7A575B7F190044E1A
:1028150012001EE0FC90F20012001EECF0780A7423
:102825000126F6500418E436F650CF750A007509EE
:1028350000AE09AF0A74FFC39F74019E402475B7AB
:10284500A575B7F190064E12001EE0FC90F400123B
:10285500001EECF0780A740126F6500418E436F6EA
:1028650050CF758F0075F51175B62075D940D2AF6B
:10287500743A90074EF022900788E0B4AA028003CC
:102885000229B9C2AF75D90075B62275F522758FC3
:102895000375B7A575B7F1740090E600F075B7A597
:1028A50075B7F1740090E800F075B7A575B7F174C8
:1028B5000090EA00F075B7A575B7F1740090EC00CB
:1028C500F0758F01750A00750900AE09AF0A74FF2E
:1028D500C39F74019E402475B7A575B7F190004E4E
:1028E50012001EE0FC90E60012001EECF0780A745F
:1028F5000126F6500418E436F650CF750A0075091E
:1029050000AE09AF0A74FFC39F74019E402475B7DA
:10291500A575B7F190024E12001EE0FC90E800127A
:10292500001EECF0780A740126F6500418E436F619
:1029350050CF750A00750900AE09AF0A74FFC39F31
:1029450074019E402475B7A575B7F190044E120029
:102955001EE0FC90EA0012001EECF0780A740126D5
:10296500F6500418E436F650CF750A00750900AE26
:1029750009AF0A74FFC39F74019E402475B7A575FE
:10298500B7F190064E12001EE0FC90EC0012001EFE
:10299500ECF0780A740126F6500418E436F650CFA8
:1029A500758F0075F51175B62075D940D2AF743A9B
:1029B50090074EF022900788E0B4AA028003022A0D
:1029C500F7C2AF75D90075B62275F522758F0375F7
:1029D500B7A575B7F1740090DE00F075B7A575B7AA
:1029E500F1740090E000F075B7A575B7F17400902B
:1029F500E200F075B7A575B7F1740090E400F075C5
:102A05008F01750A00750900AE09AF0A74FFC39FEF
:102A150074019E402475B7A575B7F190004E12005C
:102A25001EE0FC90DE0012001EECF0780A74012610
:102A3500F6500418E436F650CF750A00750900AE55
:102A450009AF0A74FFC39F74019E402475B7A5752D
:102A5500B7F190024E12001EE0FC90E00012001E3D
:102A6500ECF0780A740126F6500418E436F650CFD7
:102A7500750A00750900AE09AF0A74FFC39F74019A
:102A85009E402475B7A575B7F190044E12001EE05F
:102A9500FC90E20012001EECF0780A740126F65054
:102AA5000418E436F650CF750A00750900AE09AF73
:102AB5000A74FFC39F74019E402475B7A575B7F1CD
:102AC50090064E12001EE0FC90E40012001EECF091
:102AD500780A740126F6500418E436F650CF758F3F
:102AE5000075F51175B62075D940D2AF743A9007C7
:102AF5004EF022900788E0B4AA028003022C35C26A
:102B0500AF75D90075B62275F522758F0375B7A512
:102B150075B7F1740090D600F075B7A575B7F17467
:102B25000090D800F075B7A575B7F1740090DA007C
:102B3500F075B7A575B7F1740090DC00F0758F01DD
:102B4500750A00750900AE09AF0A74FFC39F7401C9
:102B55009E402475B7A575B7F190004E12001EE092
:102B6500FC90D60012001EECF0780A740126F6508F
:102B75000418E436F650CF750A00750900AE09AFA2
:102B85000A74FFC39F74019E402475B7A575B7F1FC
:102B950090024E12001EE0FC90D80012001EECF0D0
:102BA500780A740126F6500418E436F650CF750AF3
:102BB50000750900AE09AF0A74FFC39F74019E40FA
:102BC5002475B7A575B7F190044E12001EE0FC9070
:102BD500DA0012001EECF0780A740126F65004188B
:102BE500E436F650CF750A00750900AE09AF0A74D0
:102BF500FFC39F74019E402475B7A575B7F1900674
:102C05004E12001EE0FC90DC0012001EECF0780A6B
:102C1500740126F6500418E436F650CF758F00750A
:102C2500F51175B62075D940D2AF743A90074EF0BC
:102C350022C2AF75D90075F522750A00750900AE77
:102C450009AF0A74FFC39F74019E401F90EE0012E6
:102C5500001EE493FC90004E12001EECF0780A74FE
:102C65000126F6500418E436F650D4750A007509A5
:102C750000AE09AF0A74FFC39F74019E401F90F018
:102C85000012001EE493FC90024E12001EECF07838
:102C95000A740126F6500418E436F650D4750A0075
:102CA500750900AE09AF0A74FFC39F74019E401FEA
:102CB50090F20012001EE493FC90044E12001EECEC
:102CC500F0780A740126F6500418E436F650D475E7
:102CD5000A00750900AE09AF0A74FFC39F74019E0F
:102CE500401F90F40012001EE493FC90064E120063
:102CF5001EECF0780A740126F6500418E436F650F6
:102D0500D475F51175D940D2AF22C2AF75D900750A
:102D1500F522750A00750900AE09AF0A74FFC39F55
:102D250074019E401F90E60012001EE493FC900083
:102D35004E12001EECF0780A740126F6500418E4D1
:102D450036F650D4750A00750900AE09AF0A74FF4E
:102D5500C39F74019E401F90E80012001EE493FC7F
:102D650090024E12001EECF0780A740126F650040B
:102D750018E436F650D4750A00750900AE09AF0A95
:102D850074FFC39F74019E401F90EA0012001EE469
:102D950093FC90044E12001EECF0780A740126F69E
:102DA500500418E436F650D4750A00750900AE09CA
:102DB500AF0A74FFC39F74019E401F90EC00120080
:102DC5001EE493FC90064E12001EECF0780A740186
:102DD50026F6500418E436F650D475F51175D94029
:102DE500D2AF22C2AF75D90075F522750A007509F3
:102DF50000AE09AF0A74FFC39F74019E401F90DEA9
:102E05000012001EE493FC90004E12001EECF078B8
:102E15000A740126F6500418E436F650D4750A00F3
:102E2500750900AE09AF0A74FFC39F74019E401F68
:102E350090E00012001EE493FC90024E12001EEC7E
:102E4500F0780A740126F6500418E436F650D47565
:102E55000A00750900AE09AF0A74FFC39F74019E8D
:102E6500401F90E20012001EE493FC90044E1200F5
:102E75001EECF0780A740126F6500418E436F65074
:102E8500D4750A00750900AE09AF0A74FFC39F74B3
:102E9500019E401F90E40012001EE493FC90064E34
:102EA50012001EECF0780A740126F6500418E43678
:102EB500F650D475F51175D940D2AF22C2AF75D988
:102EC5000075F522750A00750900AE09AF0A74FF91
:102ED500C39F74019E401F90D60012001EE493FC10
:102EE50090004E12001EECF0780A740126F650048C
:102EF50018E436F650D4750A00750900AE09AF0A14
:102F050074FFC39F74019E401F90D80012001EE4F9
:102F150093FC90024E12001EECF0780A740126F61E
:102F2500500418E436F650D4750A00750900AE0948
:102F3500AF0A74FFC39F74019E401F90DA00120010
:102F45001EE493FC90044E12001EECF0780A740106
:102F550026F6500418E436F650D4750A00750900B3
:102F6500AE09AF0A74FFC39F74019E401F90DC0039
:102F750012001EE493FC90064E12001EECF0780A37
:102F8500740126F6500418E436F650D475F511751B
:102F9500D940D2AF22E51464046006E59964FF6068
:102FA500028031A20F4004D20F8027E51460087417
:102FB500E62514900023F0E513600874F0251390BE
:102FC5000023F0E514B4010280FE751400751300AA
:102FD500C20F8002C20FE5149038F5F828287375E2
:102FE5001400E599B4FF03751301E599B4FE037563
:102FF5001302E599B4FD03751303E599B4FC037554
:103005001304E599B4FA03751305E599B4FB067540
:103015001401120464E599B4F906751404120464E4
:10302500E599D394E54007E599C394F040028016ED
:103035008599157514027E017F00E515C394E61286
:103045003FE18E0D8F0E900786E4F0A3F0E599D34E
:1030550094C44007E599C394E640028028859915F4
:1030650075140374E5C39515F50E750D00AE0DAF1A
:103075000E90395212002EE493F87401939007864E
:10308500C8F0A3C8F0D299023509900786E0FEA3DF
:10309500E0FFEFC39400EE94054009EFD394FFEEF3
:1030A50094064013900786E0FEA3E0FF90004E12C1
:1030B500001EE599F0800385996B90078612000E36
:1030C500900786E0FEA3E0FFEFB40106EEB4070229
:1030D500800302331990074EE0B43C0280030233AB
:1030E50019A20AB35005A20BB3400302320CC29CCD
:1030F50090007AE090078CF0900057E090078DF0F3
:10310500900062E090078EF0900063E090078FF0EA
:10311500900074E0900790F090007CE0900791F0AB
:1031250090007DE0900792F0900080E0900793F08A
:10313500900081E0900794F090013AE0900795F0B7
:1031450090013BE0900796F090013CE0900797F0E6
:10315500900090E0900798F0900091E0900799F02A
:10316500900092E090079AF0900093E090079BF012
:10317500900094E090079CF0900095E090079DF0FA
:10318500900096E090079EF0900097E090079FF0E2
:10319500900099E09007A0F090009AE09007A1F0C8
:1031A50090009BE09007A2F090009CE09007A3F0B0
:1031B5007400900082F01200AC74AB900788F01296
:0A31C500269374AA900788F0E558DD
:0638F500022FE402308FF7
:1031CF00903916F8282873801212273E800D122886
:0B31DF007C80081229BA8003122AF835
:0F3916000231D60231D80231DD0231E20231E74F
:1031EA00900788E4F090013AE0700C90013BE0709F
:1031FA000690013CE060028004C20A8002D20A0200
:10320A00330EC29C900078E0900789F090005EE04F
:10321A0090078AF090005FE090078BF090007AE0C8
:10322A0090078CF0900057E090078DF0900062E0D4
:10323A0090078EF0900063E090078FF0900074E0A2
:10324A00900790F090007CE0900791F090007DE06C
:10325A00900792F0900080E0900793F0900081E050
:10326A00900794F090013AE0900795F090013BE0C6
:10327A00900796F090013CE0900797F0900090E05C
:10328A00900798F0900091E0900799F0900092E0F2
:10329A0090079AF0900093E090079BF0900094E0DA
:1032AA0090079CF0900095E090079DF0900096E0C2
:1032BA0090079EF0900097E090079FF0900099E0A9
:1032CA009007A0F090009AE09007A1F090009BE090
:1032DA009007A2F090009CE09007A3F07400900081
:1032EA0082F074AB900788F012269374AA9007882C
:1032FA00F012273E12287C1229BA122AF8D29C759B
:10330A0099FB80FED29C7514007513007599FB0217
:10331A003509900786E0FEA3E0FFEF4E7006859917
:10332A0010750F00900786E0FEA3E0FF74016F4E50
:10333A00701BAC0FAD10AA0DAB0EED2BFBEC3AFADD
:10334A008A068B0790004E12001EE599F0900786B8
:10335A0012000E900786E0FEA3E0FF74026F4E7023
:10336A000C1200AC85159975140075130002350905
:10337A00900786E0FEA3E0FF90004E12001EE5993A
:10338A00F090078612000E900786E0FEA3E0FFACDD
:10339A000DAD0E8F028E038C068D0790398A1200AE
:1033AA002EE493F9740193FEEAD39EEB99400985C2
:1033BA001599751400751300023509900786E0FE09
:1033CA00A3E0FF90004E12001EE599F090078612C6
:1033DA00000E900786E0FEA3E0FFEFB40006EEB40D
:1033EA000102800302350990001CE0D394C7400B08
:1033FA0090001CE0C394C8F516801A90001CE0D314
:10340A009463400B90001CE0C39464F51680069008
:10341A00001CE0F516E51675F002A4FFAEF08F6AFF
:10342A00EF90004E123FF9EFFCE0FDEC90005112D4
:10343A003FF9EDFCE0FDEC2DB5160280030234FBEA
:10344A000FEF90004E123FF9E56AFFE0FCEF9000A3
:10345A0052123FF9ECFFE0FCEFC39CB51602800361
:10346A000234FBE56A900050123FF9E56AFFE0FC7E
:10347A00EF900053123FF9ECFFE0FCEF2CB5167108
:10348A00E56A900054123FF9E0C3951690079DF043
:10349A00E56A900055123FF9E0C3951690079EF031
:1034AA00E56A900058123FF9E0C3951690079FF01D
:1034BA00E56A900059123FF9E0C395169007A0F00B
:1034CA00E56A90005A123FF9E0C395169007A1F0F9
:1034DA00E56A90005B123FF9E0C395169007A2F0E7
:1034EA001226097599F97518647517001225C58091
:0F34FA00FE7599FF7518647517001225C580FEC1
:0938FB0002331C02337A0233C5CA
:1035090022E513903904F828287302364A90078671
:10351900E0FEA3E0FF90001212001EE0F59990076B
:103529008612000E900786E0FEA3E0FF74116F4E2D
:10353900700375130002364A85619902364A90076D
:1035490086E0FEA3E0FF90004E12001EE0F599EF21
:10355900B40107EEB4070375130090078612000E35
:0735690002364A900787E0DB
:0F39040002351302351602354102354702356C84
:10357000903925F828287385249902363F852A99A1
:1035800002363F85449902363F85479902363F858A
:10359000519902363F855F9902363F85569902362A
:1035A0003F85589902363F756D00900069E07006BE
:1035B000900068E060028016A2A44006E56D440415
:1035C000F56DA2A54006E56D4402F56D801A9000E8
:1035D0004AE0B40106E56D4410F56D900049E0B491
:1035E0000106E56D4420F56DA207B34006E56D4484
:1035F00001F56DA209B34006E56D4408F56D856DD2
:1036000099803CA210B340077599FAC2108017A2A6
:103610000CB3400575990F800B900023E0F599904D
:103620000023E4F0C20C80178542998012854B99E3
:0F363000800D85469980087599FC8003751300FD
:1039250002357702357D02358302358902358F02EE
:10393500359502359B0235A10235A70236030236BD
:0D3945002802362D02363202363702363C9B
:0B363F0090078612000E800312004866
:0339130002364732
:10364A002290006BE0B4010385241190006BE0B472
:10365A000203852A1190006BE0B40303854411909C
:10366A00006BE0B4040385471190006BE0B40503D6
:10367A0085511190006BE0B4060385561190006BDA
:10368A00E0B4070385581190006CE0FE90006DE0ED
:10369A00C39E500302372190006BE0D39404402C60
:1036AA0090006CE0D39511500990006DE0C395111C
:1036BA0050028002D20090006CE0D395115009901C
:1036CA00006DE0C395115002C200804990006BE082
:1036DA00B4041890006DE0C395115002D200900016
:1036EA006CE0D395114002C200802A90006CE0C3BE
:1036FA009511500990006DE0D3951150028002D2C5
:10370A000090006CE0D39511500990006DE0C395CC
:10371A00115002C200807E90006BE0D39404402CCA
:10372A0090006CE0C39511400990006DE0D39511AB
:10373A0040028002C20090006CE0C39511400990DB
:10374A00006DE0D395114002D200804990006BE0F1
:10375A00B4041890006CE0C395115002C2009000A6
:10376A006DE0D395114002D200802A90006CE0C32C
:10377A009511400990006DE0D395114002D2009056
:10378A00006CE0D39511400990006DE0C39511409B
:10379A00028002C2002290006EE0B4010385241167
:1037AA0090006EE0B40203852A1190006EE0B40323
:1037BA000385441190006EE0B4040385471190001C
:1037CA006EE0B4050385511190006EE0B4060385DE
:1037DA00561190006EE0B4070385581190006FE00F
:1037EA00FE900070E0C39E500302387690006EE0AF
:1037FA00D39404402C90006FE0D3951150099000A7
:10380A0070E0C3951150028002D20290006FE0D39B
:10381A0095115009900070E0C395115002C20280C0
:10382A004990006EE0B40418900070E0C3951150FE
:10383A0002D20290006FE0D395114002C202802AA0
:10384A0090006FE0C395115009900070E0D3951174
:10385A0050028002D20290006FE0D3951150099075
:10386A000070E0C395115002C202807E90006EE0A3
:10387A00D39404402C90006FE0C395114009900046
:10388A0070E0D3951140028002C20290006FE0C33B
:10389A0095114009900070E0D395114002D2028040
:1038AA004990006EE0B4041890006FE0C39511507F
:1038BA0002C202900070E0D395114002D202802A1F
:1038CA0090006FE0C395114009900070E0D3951104
:1038DA004002D20290006FE0D39511400990007027
:0B38EA00E0C3951140028002C20222E0
:093FF9002582F5825002058322A5
:10002E00EF2F500205832582F582E5833E2EF58360
:01003E00229F
:08000300C3EF9DFFEE9CFE22FD
:08003F000806B60002180622B3
:0D000E00A3E004F07006123FEFE004F022C2
:08400B000816B6FF0218162288
:0E3FD300048007C3CE13CECF13CFD5E0F62265
:103E8100BC000FBE0008ED8FF084FFADF022E4FE10
:103E9100FF22BE000DEF60FE54F0606F20E70302C9
:103EA1003F37EAC0E0EBC0E078017A0075F001EE3F
:103EB10020E710EF25E0FFEE33FE0AC5F023C5F041
:103EC10030E7F0EA5407F9096A7A007B00600108DB
:103ED100C3EC9E40167004ED9F4010ED9FFDEC9EDB
:103EE100FCE5F0CA4ACA03F5F08005E5F003F5F0F8
:103EF100C3EE13FEEF13FFD9D77908CACBCAD8D0C6
:103F0100EAFEEBFFD0E0FBD0E0FA22EC8FF084FC7C
:103F1100ED54F045F0C48FF084FEEDC454F045F04B
:103F2100C48FF084FDEEC4FE54F02DFFEE540F3C1F
:103F3100FEADF07C0022790078008FF0EC7E082045
:103F4100E70DC3CD33CD33C933C9C833C8DEF084DF
:103F510049F9E5F08FF0BE00E6FD7C00E9FFE8FEDF
:013F6100223D
:0E3FE100F88FF0A4FFE5F0CE88F0A42EFE22AB
:103FB300600D782B023FBD007830D8FED5E0F822A3
:103FC300EEC0E07E00123E81EFFDEEFCD0E0FE226B
:03000B00023F624F
:03001B00023F7D24
:03002B00023F98F9
:03000000024002B9
:0940020075817175D000020712EE
:0B001E00E5822FF582E5833EF583228A
:0A3FEF000582D58202158315822297
:103F6200C0E0C0F0C083C082C0D075D00012070785
:103F7200D0D0D082D083D0F0D0E032C0E0C0F0C048
:103F820083C082C0D075D00012070AD0D0D082D0B0
:103F920083D0F0D0E032C0E0C0F0C083C082C0D095
:103FA20075D00012070DD0D0D082D083D0F0D0E0EF
:013FB20032DC
:00000001FF
